:0200000480007A
:10000000970000009380C004130E100093001000AE
:100010001301300093802000639A2002130E200009
:100020009300300117010000130101026F0040002E
:10003000232011000F100000130A8000130AFAFF9A
:10004000E31E0AFE6F0080006F000001370110F010
:10005000130141F22320C101370110F0130101F215
:100060002320010013000000130000001300000013
:100070001300000013000000130000000000000047
:04008000000000007C
:00000001FF
